:020000040000FA
:10040000BFFFDFFFFFFFFFFFFFFFFFFFFFFFFFFF5C
:10041000FFFFFFFFFFFFFFFFFFFFFFFFFFFFFFFFEC
:10042000FFFFFFFFFFFFFFFFFFFFFFFFFFFFFFFFDC
:10043000FFFFFFFFFFFFFFFFFFFFFFFFFFFFFFFFCC
:10044000FFFFFFFFFFFFFFFFFFFFFFFFFFFFFFFFBC
:10045000FFFFFFFFFFFFFFFFFFFFFFFFFFFFFFFFAC
:020000040000FA
:1080000098370020258300002D830000458D000057
:10801000318300003383000035830000000000003E
:108020000000000000000000000000006582000069
:108030003983000000000000C1820000699A00003E
:10804000B58D0000C58D0000D58D0000E58D0000C8
:10805000F58D0000058E0000158E0000258E0000B5
:10806000358E0000458E0000558E0000658E0000A4
:10807000758E0000858E0000958E0000A58E000094
:10808000E5890000F98900003F8300003F8300007C
:108090003F8300003F8300003F8300003F830000D8
:1080A0002D8A0000438A0000598A00006F8A000070
:1080B000858A0000AF8A0000C58A00003F83000067
:1080C0003F8300003F8300003F8300003F830000A8
:1080D0003F8300003F8300003F8300003F83000098
:1080E0003F8300003F8300003F8300003F83000088
:1080F0003F8300003F8300003F8300003F83000078
:108100003F8300003F8300003F8300003F83000067
:108110003F8300003F8300003F8300003F83000057
:108120003F8300003F8300003F8300003F83000047
:108130003F8300003F8300003F8300003F83000037
:108140003F8300003F8300003F8300003F83000027
:108150003F8300003F8300003F8300003F83000017
:108160003F8300003F8300003F8300003F83000007
:108170003F8300003F8300003F8300003F830000F7
:108180003F8300003F8300003F8300003F830000E7
:108190003F8300003F8300003F8300003F830000D7
:1081A0003F8300003F8300003F8300003F830000C7
:1081B0003F8300003F8300003F8300003F830000B7
:1081C0003F8300003F8300003F8300003F830000A7
:1081D0003F8300003F8300003F8300003F83000097
:1081E0003F8300003F8300003F8300003F83000087
:1081F0003F8300003F8300003F8300003F83000077
:108200003F8300003F8300003F8300003F83000066
:108210003F8300003F830000CD8F00003F830000BC
:108220009D9100003F8300003F8300003F830000DA
:108230003F8300003F8300003F8300003F83000036
:108240003F8300003F8300003F8300003F83000026
:10825000DFF80CD000F0ECF800480047F5AD000066
:10826000983700202C4B19680868B0E8F04F80F36D
:108270000988BFF36F8F4FF0000080F311887047BB
:108280000000000008480068006880F308884FF08C
:10829000000080F3148862B661B6BFF34F8FBFF35E
:1082A0006F8F00DF00BF00BF08ED00E0DFF80C00BB
:1082B000016841F470010160704700BF88ED00E083
:1082C000EFF30980BFF36F8F134B1A681EF0100F86
:1082D00008BF20ED108A20E9F04F106009B44FF07C
:1082E000500080F31188BFF34F8FBFF36F8F04F0FE
:1082F000FDFB4FF0000080F3118809BC1968086885
:10830000B0E8F04F1EF0100F08BFB0EC108A80F3F9
:108310000988BFF36F8F70476882FF1FEFF30580F6
:10832000704700000648804706480047FEE7FEE722
:10833000FEE7FEE7FEE7FEE7FEE7FEE7FEE7FEE715
:10834000699B0000518200002DE9F05F0546002086
:1083500092469B4688460646814640241BE02846B6
:1083600041464746224600F053F853465A46C01A43
:10837000914110D311461846224600F016F82D1AE6
:1083800067EB01084F4622460120002100F00DF85E
:1083900017EB00094E41201EA4F10104DFDC484622
:1083A00031462A464346BDE8F09F202A04DB203AA6
:1083B00000FA02F1002070479140C2F1200320FA38
:1083C00003F319439040704740EA01039B0703D031
:1083D00009E008C9121F08C0042AFAD203E011F804
:1083E000013B00F8013B521EF9D27047D2B201E0C6
:1083F00000F8012B491EFBD270470022F6E710B5AA
:1084000013460A4604461946FFF7F0FF204610BD02
:10841000202A04DB203A21FA02F00021704721FAD9
:1084200002F3D040C2F12002914008431946704740
:10843000064C074D06E0E06840F0010394E80700B1
:1084400098471034AC42F6D3FFF706FF50DC00002B
:1084500070DC000030B58C1810F8012B12F00F03FF
:1084600001D110F8013B120906D110F8012B03E0ED
:1084700010F8015B01F8015B5B1EF9D101E001F826
:10848000013B521EFBD1A142E6D3002030BD08B50E
:108490000021009102E00099491C0091009981425D
:1084A000F9D308BD014604480078084008B101200E
:1084B00070470020FCE700003C40054070B50446D2
:1084C000002564B91648007800F00700052801D19E
:1084D000AD1F22E001201249091D08701DE010485F
:1084E000DA300068C0F3C01030B94FF48051082072
:1084F00000F073F8054605E04FF48051012000F0CC
:108500006CF805464DB900200549091D08704FF467
:108510008051202000F061F80546284670BD00001B
:108520002640054070B5044614B96FF0020514E00A
:108530002079C1090A48006861F3C710084908603A
:1085400060680860207820B90120FFF7B7FF054672
:1085500003E00020FFF7B2FF0546284670BD00008B
:10856000004105400146002009B9C01E22E000225A
:108570004A604A6822F080024A604A6822F0030298
:108580004A6013234A6863F310224A604A6822F063
:10859000704202F180524A604A6822F0706202F131
:1085A00080724A604A6822F4700202F580124A60C2
:1085B00001220A70704770B504460D4629462046D0
:1085C00001F086F901F06AFA70BD10B50446204644
:1085D00001F0E8F901F062FA10BD18B503460A4649
:1085E000002000906FF0070409E01846FFF75AFFDB
:1085F000012801D1002405E00098401C009000985B
:108600009042F2D900BF204618BD000070B5044664
:108610000025F4B91548007800F00700032801D1BF
:10862000AD1F20E01148DA300068C0F3C01058B91F
:108630000E48001D007810B96FF0050513E0012009
:108640000A490C3108700EE0012008490C3108700D
:1086500009E0002005490C3108704FF480510820D2
:10866000FFF7BBFF0546284670BD000026400540C9
:1086700070B5044614B96FF0020514E0E0780B49B8
:108680000870607840F08000A178084308490870BD
:10869000207820B90120FFF7B9FF054603E000204C
:1086A000FFF7B4FF0546284670BD0000A240054014
:1086B00050CC04400146002009B9C01E06E001224A
:1086C0000A7000228A704A700522CA707047000042
:1086D000024909680143014A1160704724040140BE
:1086E000012805D10749084A1160C943116007E014
:1086F00005491831096841F48031034A1832116084
:108700007047000067452301040401400146044806
:1087100000680840884201D1012070470020FCE732
:10872000200401402DE9FF5F80468946164600205F
:108730000390B008019006F0030A4F464546002416
:1087400040F23F10FFF7C4FF3848006800F4702083
:1087500002903648006820F4702034490860081DF3
:10876000006820F00700401C091D08601FE001CFD1
:1087700001C52F48006AC0F302612E480068C84056
:1087800044F62061B0FBF1F04FF48071009001FAE3
:1087900004F0009900F00EF910F1080F02D16FF00B
:1087A00004000390102101FA04F0FFF791FF0198F3
:1087B000411E01910028DAD1BAF1000F27D0D7F875
:1087C00000B04FEACA01401E884040EA0B0B45F852
:1087D00004BB1748006AC0F3026116480068C8402D
:1087E00044F62061B0FBF1F04FF48071009001FA83
:1087F00004F0009900F0DEF810F1080F02D16FF0DC
:1088000004000390102101FA04F0FFF761FF07480C
:10881000006820F47020029901F470210843034994
:108820000860039804B0BDE8F09F00001804014000
:1088300000400540902B00202DE9F05F05460C46D6
:1088400016466FF002092F46B0464FF4807AF4B115
:108850001048006AC0F302610F480068C84044F63F
:108860002061B0FBF1FB5946504600F0A3F860B917
:1088700005E017F8010B04F8010BA8F10108B8F1A5
:10888000000FF6D14FF0000901E06FF004094846EF
:10889000BDE8F09F00400540902B00202DE9F041FD
:1088A0000446002640F23F10FFF712FF2048006800
:1088B00000F470271E48006820F470201C490860EE
:1088C0000025081D006820F00700001D091D086034
:1088D000002020601748006AC0F302611648006853
:1088E000C8403221B0FBF1F84FF4807101FA05F075
:1088F000414600F05FF810F1080F00D16E1F102103
:1089000001FA05F0FFF7E4FE0948001D006820F0B9
:1089100007000749091D0860081F006820F470203F
:1089200007F470210843024908603046BDE8F08131
:108930001804014000400540902B00200146002211
:108940000F48006861F303000D4B186010E0521CE3
:108950000C48006AC0F302630B480068D84044F634
:108960002063B0FBF3F0904202D26FF00700704733
:108970000348006800F00F008842E8D10020F6E7C5
:108980001804014000400540902B002030B50246FD
:1089900002F01F00064B1B6801248440A34301FA28
:1089A00000F4012585402C402343014C236030BD59
:1089B0009005014018B503460A46002000900024A7
:1089C00008E00098401C00900098904202D96FF097
:1089D000070404E01846FFF799FE0128F1D100BF13
:1089E000204618BD10B5012000F080F8012801D103
:1089F00000F074F810BD000010B5022000F076F809
:108A0000012805D103A001F023F9022000F066F847
:108A100010BD0000455854494E545F434830312042
:108A2000696E74657272757075740A0010B54FF4D2
:108A3000807000F05BF8012802D1000200F04EF8CF
:108A400010BD10B54FF4007000F050F8012802D1AD
:108A5000400200F043F810BD10B54FF4806000F004
:108A600045F8012802D1800200F038F810BD10B599
:108A70004FF4006000F03AF8012802D1C00200F083
:108A80002DF810BD10B54FF4805000F02FF80128DC
:108A90000CD10103042000F0F9F84FF480510220BA
:108AA00000F0F4F84FF4805000F018F810BD10B545
:108AB0004FF4005000F01AF8012802D1400300F0F2
:108AC0000DF810BD10B54FF4804000F00FF80128EC
:108AD00002D1800300F002F810BD00000249896D48
:108AE0000143014A91657047001005400146044862
:108AF000406D084008B1012070470020FCE70000ED
:108B000000100540012905D1054A52688243044BF3
:108B10005A6004E0024A52680243014B5A607047AF
:108B2000008004402DE9F04705460F469046002698
:108B3000B146002421E0285D5A281DD1601C295C23
:108B4000A01C285C01EB002086B2A019401CB84292
:108B500012D2B11E281901F000FBA119891E6A5C0E
:108B6000A119491E695C02EB0121884204D14FF032
:108B70000109A8F8004006E0641CF81FA04202D9D1
:108B8000B9F1000FD7D000BFB9F1000F02D100201A
:108B9000BDE8F0873046FBE730B503460C460021C0
:108BA00015E001258D4025407DB10A4D05EB83156B
:108BB00005EB8100012A04D1058845F400450580B4
:108BC00003E00588C5F30E0505804D1CE9B21029A8
:108BD000E7D330BD003C05402DE9F04104460F4687
:108BE00000200AB9C01E4CE0002148E04FF0010C03
:108BF0000CFA01FC0CEA070CBCF1000F3BD0B2F8F8
:108C000000C0B2F802804CEA080CB2F804804CEACA
:108C1000080CB2F806804CEA080CB2F80A804CEA5C
:108C2000080CB2F80E804CEA080CB2F810804CEA3E
:108C3000080CB2F808804CEA080545F27723B2F830
:108C400014C04CEA050543F40043B2F812C04CEAE4
:108C5000050543F48063DFF830C00CEB841C0CEB9B
:108C60008106B6F800C02CEA030C05EA03084CEABA
:108C7000080CA6F800C001F1010C0CF0FF0110294E
:108C8000B4D3BDE8F0810000003C05400246054B2E
:108C900003EB0210B0F80008084008B1012070474B
:108CA0000020FCE70030054010B5044B102404FB05
:108CB000003213880B43138010BD00000A380540B2
:108CC00030B5034600200BE0012585400D402DB155
:108CD000054D05EB831505EB80042280451CE8B2A9
:108CE0001028F1D330BD0000023C054010B5044B04
:108CF000102404FB003213880B43138010BD0000C6
:108D0000083805400549098848F6FF72114000F40B
:108D1000E0421143014A118070470000F83B0540D2
:108D20000146002009B9C01E0BE000220A804A80DB
:108D3000CA808A828A810A814A81CA810A828A809B
:108D40004A82704700BFFEE730B50146002009B9EE
:108D5000C01E2AE0B1F902300F2B02DD6FF00200D5
:108D600023E04B88114C042515FB03421368C3F321
:108D7000080340F2FF14A34208D10B881360B1F935
:108D800002400B4D4B6845F824300EE00B88146808
:108D9000C4F30804A34206D1B1F90240044D4B6864
:108DA00045F8243001E06FF0010030BD5C10054053
:108DB000F4ACFF1F10B502490868804710BD0000E1
:108DC000F4ACFF1F10B502494868804710BD000091
:108DD000F4ACFF1F10B502498868804710BD000041
:108DE000F4ACFF1F10B50249C868804710BD0000F1
:108DF000F4ACFF1F10B502490869804710BD0000A0
:108E0000F4ACFF1F10B502494869804710BD00004F
:108E1000F4ACFF1F10B502498869804710BD0000FF
:108E2000F4ACFF1F10B50249C869804710BD0000AF
:108E3000F4ACFF1F10B50249086A804710BD00005E
:108E4000F4ACFF1F10B50249486A804710BD00000E
:108E5000F4ACFF1F10B50249886A804710BD0000BE
:108E6000F4ACFF1F10B50249C86A804710BD00006E
:108E7000F4ACFF1F10B50249086B804710BD00001D
:108E8000F4ACFF1F10B50249486B804710BD0000CD
:108E9000F4ACFF1F10B50249886B804710BD00007D
:108EA000F4ACFF1F10B50249C86B804710BD00002D
:108EB000F4ACFF1F10B5044604F0010048B100BF38
:108EC00040F223101A49086043F21020086000BFE6
:108ED00000BF04F0020028B100BF1648164908611F
:108EE00000BF00BF04F0040030B100BF4AF20150DF
:108EF0001249088000BF00BF04F0100018B14AF208
:108F0000085000F04FFB04F0400018B14AF2035043
:108F100000F048FB04F0800040B100BF7720084912
:108F2000086007490831086000BF00BF10BD00009D
:108F3000000401400100A5A500800440FC3B054061
:108F40000408054010B5044604F0010028B100BF34
:108F500000201949086000BF00BF04F0020028B1DA
:108F600000BF16481649086100BF00BF04F00400A6
:108F700030B100BF4FF425401249088000BF00BF48
:108F800004F0100018B14AF2085000F0FDFA04F0A5
:108F9000400018B14AF2035000F0F6FA04F08000E5
:108FA00040B100BF762008490860074908310860D1
:108FB00000BF00BF10BD0000000401400000A5A5D7
:108FC00000800440FC3B05400408054030B59FB0DC
:108FD000002501215D4800F0CFFA012845D101218B
:108FE0005A4800F0A7F95AA000F032FE04AA402126
:108FF000564800F0C1F9002837D1002405E00EA83A
:10900000015D5AA000F024FE641C082CF7DB0598D3
:10901000C0B28DF800000498019008208DF801007E
:10902000DDE90E01CDE902010498B0F5F66F07D134
:1090300000234F4A04A94F48006803F0F3FE06E0FE
:1090400002234B4A69464C48006803F0EBFE00BF20
:109050004748006838B14FF0805048490860BFF376
:109060004F8FBFF36F8F00BF00BF0421374800F060
:1090700083FA012803D10421344800F05BF9102160
:10908000324800F079FA012845D110212F4800F02C
:1090900051F93BA000F0DCFD04AA41212B4800F06F
:1090A0006BF9002837D1002405E00EA8015D2FA040
:1090B00000F0CEFD641C082CF7DB0598C0B28DF8DB
:1090C00000000498019008208DF80100DDE90E01F0
:1090D000CDE902010498B0F5F66F07D10223244AC6
:1090E00004A92448006803F09DFE06E00223204AFC
:1090F00069462148006803F095FE00BF1C480068DF
:1091000038B14FF080501D490860BFF34F8FBFF357
:109110006F8F00BF00BF40210C4800F02DFA0128DE
:1091200007D14021094800F005F92946074800F019
:1091300003F94FF40021054800F01EFA012803D17D
:10914000C104024800F0F6F81FB030BD00900240A4
:109150005278204649464F5F30206E6577206D6516
:1091600073736167652D3E0D0A00000025782000AD
:109170003482FF1F2882FF1F2C82FF1F04ED00E0B6
:109180005278204649464F5F31206E6577206D65E5
:1091900073736167652D3E0D0A00000030B59FB006
:1091A00000250121504800F0E7F9012838D10121BC
:1091B0004D4800F0BFF84DA000F04AFD04AA402140
:1091C000494800F0D9F858BB002405E00EA8015D1D
:1091D0004DA000F03DFD641C082CF7DB0598C0B2E3
:1091E0008DF800000498019008208DF80100DDE959
:1091F0000E01CDE902010223444A69464448006851
:1092000003F010FE00BF4148006838B14FF08050B5
:1092100040490860BFF34F8FBFF36F8F00BF00BF9F
:109220000421314800F0A8F9012803D104212E4877
:1092300000F080F810212C4800F09EF9012838D168
:109240001021294800F076F833A000F001FD04AAAF
:109250004121254800F090F858BB002405E00EA8F5
:10926000015D29A000F0F4FC641C082CF7DB0598D4
:10927000C0B28DF800000498019008208DF801001C
:10928000DDE90E01CDE902010223204A69462048AA
:10929000006803F0C7FD00BF1C48006838B14FF0FC
:1092A00080501C490860BFF34F8FBFF36F8F00BF22
:1092B00000BF40210C4800F05FF9012807D1402190
:1092C000094800F037F82946074800F035F84FF410
:1092D0000021054800F050F9012803D1C1040248DB
:1092E00000F028F81FB030BD0094024052782046AC
:1092F00049464F5F30206E6577206D6573736167F7
:10930000652D3E0D0A000000257820003882FF1FE1
:109310003082FF1F04ED00E05278204649464F5F3F
:1093200031206E6577206D6573736167652D3E0D25
:109330000A00000001657047C0F8D01070470000B7
:109340000146AC31486C4FF6FC731840084BC2180C
:1093500008684FF6FC731840054B1844121A086948
:10936000AC39C0F30220034B185CB2FBF0F070473D
:1093700000B0024048DC00002DE9FC5F04460F46C7
:1093800015464FF000080020009083466FF0020958
:10939000002D7CD08146402F2ED1D4F8A00000F4BF
:1093A000FE0008B96FF00209B9F1000F06D1D4F838
:1093B000A40000F07F0008B96FF00809B9F1000FB0
:1093C0006CD1A0346068C0F3052B20684FF6FC71A7
:1093D0000840664900EB0108E06900F007006449B5
:1093E000085C1BFB0088E069A03C00F00700083027
:1093F0006049085C009051E0412F2ED1D4F8B000B4
:1094000000F4FE0008B96FF00209B9F1000F06D1AF
:10941000D4F8B40000F07F0008B96FF00809B9F182
:10942000000F3BD1B0346068C0F3052B20684FF6C5
:10943000FC7108404D4900EB0108E068C0F30210E0
:109440004B49085C1BFB0088E068B03CC0F302108D
:1094500008304849085C009020E02046FFF770FF84
:10946000B84202D86FF0020918E054F8AC0F4FF67A
:10947000FC7108403D4900EB01082069C0F302205F
:109480003B49085C07FB00882069AC3C00E057E0E2
:10949000C0F3022008303749085C0090B9F1000F92
:1094A00061D146463068C0F380706860686820B952
:1094B0003068C0F38A40286003E0306820F06040E4
:1094C00028603068C0F34070A8603068C00F286121
:1094D00008F10406308880B2E8613068C0F30340C8
:1094E000E8602449E868085CA866A96E0098814293
:1094F00001D90098A8663068C0F3005068613068F0
:10950000C0F34050A8613068C0F30660286230683C
:10951000C00F686208F1080601964FF0000A08E0E3
:10952000019810F80A1005F1280000F80A100AF155
:10953000010AA86E5045F3D8402F02D1C4F8A8B054
:1095400011E0412F02D1C4F8B8B00CE0202F04D2B2
:109550000120B840C4F8980005E007F01F01012081
:109560008840C4F89C004846BDE8FC9F00B002401B
:1095700048DC000038DC000002460020136D0B4080
:1095800003B101207047000004490988814341F478
:109590002541034AA2F8FE1370470000FE43054030
:1095A00000400540034909880143034AA2F8FE131D
:1095B00070470000FE4305400040054000B587B0FD
:1095C0000020ADF8060001AA4FF480610220FFF7E9
:1095D00003FB07B000BD00B587B00020ADF8060062
:1095E00001AA4FF48051FFF7F7FA07B000BD00B5AC
:1095F00087B00220ADF806000420ADF8080001AAEB
:1096000001020220FFF7E8FA07B000BD00B587B0FD
:109610000220ADF806000420ADF8080001AA81027E
:109620000020FFF7D9FA07B000BD012904D1426834
:1096300042F04002426003E0426822F04002426091
:10964000704730B502466FF00200A9B38B68082B53
:1096500003D1CB68B3F5805F2ED00B68012B06D108
:109660008B6823B94B693BB34B69022B24D0D1E9FA
:10967000003423438C6823434C6A2343CC68234340
:109680000C69234353600C8B04F470448B6A2343AE
:109690004FF203042340D4684FF20305AC43234345
:1096A000D3600C6A4B692343CC6923430C7E04F0DE
:1096B0000C0423439361002030BD012A03D1436889
:1096C0000B43436002E043688B43436070470146AD
:1096D0000868704710B54048FFF7F9FF3F49087028
:1096E0003F480088401C80B23D490880B0F5007FAB
:1096F00006D10020088000213A48006803F02DFCC4
:1097000039480078C0B9354800785A2814D101206A
:109710003549087031490A7834490888411C334B6F
:109720001980334909880144324B5A5400212D488D
:10973000006803F012FC4DE02C480088012803D09B
:109740002A48008802281ED124490A782749088817
:10975000411C264B1980264909880144254B5A543F
:1097600022480088032835D1194621480088401C2A
:10977000095C1A461E480088801C105C01EB002022
:109780001D49088026E0194800881B49098888423D
:1097900019DA12490A7815490888411C134B1980B7
:1097A000134909880144134B5A5410480088124940
:1097B000098888420ED100200C4908800E49088093
:1097C0000949087006E00020084908800A49088015
:1097D0000549087010BD0000000002406282FF1FB2
:1097E0006682FF1F5C82FF1F6182FF1F5882FF1F7E
:1097F0005482FF1FF1AAFF1F6482FF1F01466FF012
:10980000020099B100220A604A6008228A600022A0
:10981000CA600A614A614FF440528A614FF4806223
:10982000CA6100220A624A628A6200207047000010
:1098300010B50B480088FF2804DDBB21094800F063
:1098400017F80CE006480488601C054A108006489A
:1098500000882044054A115C024800F009F810BD58
:109860005082FF1F000002405282FF1FF1A8FF1F1D
:109870000160704710B500F0010353B1134B1B6832
:1098800062F30203114C236023461B6861F3061345
:10989000236000F0020353B10C4B1B6862F31243C8
:1098A0000A4C236023461B6861F31653236000F0C3
:1098B000040353B1054B1B6862F31A63034C236026
:1098C00023461B6861F31E73236010BD000805402A
:1098D0002DE9FF4104460D4600262E4800680390FE
:1098E0002C48406802902B48806801902948C06845
:1098F00000902948007800F00700052816D10126BD
:10990000264824490860C01248608860C860224820
:109910002638006AC0F3026121480068C8404CF252
:109920005031B0FBF1F73846FEF7B1FD1A48263842
:10993000006AA04305EA0401084317492639086272
:109940000846006AC0F3026115480068C8404CF23E
:109950005031B0FBF1F73846FEF799FD012E17D1D3
:109960000C49039808600298486001988860009844
:10997000C86009482638006AC0F3026108480068D8
:10998000C8404CF25031B0FBF1F73846FEF77FFD8E
:10999000BDE8FF8100800440264005400EFAFFFF2D
:1099A000902B00207FB5044600252B4800680390CB
:1099B0002948406802902848806801902648C0687D
:1099C00000902648007800F00700052801D0052CFB
:1099D00016D10125224820490860C01248608860DD
:1099E000C8601E482638006AC0F302611D4800683E
:1099F000C8404CF25031B0FBF1F63046FEF747FD5F
:109A00001648047015482638006AC0F302611548EC
:109A10000068C8404CF25031B0FBF1F63046FEF71A
:109A200036FD012D17D10C49039808600298486053
:109A3000019888600098C86008482638006AC0F31A
:109A4000026108480068C8404CF25031B0FBF1F6A2
:109A50003046FEF71CFD7FBD0080044026400540D7
:109A60000EFAFFFF902B002010B500BF502080F3AE
:109A70001188BFF34F8FBFF36F8F00BF03F018FD46
:109A800018B14FF080500449086000BF002080F3F7
:109A9000118800BF10BD000004ED00E070B52B4D33
:109AA0002D6805F001051DB1294D2A4E356002E0F3
:109AB000294D284E3560294D2D7805F007000628E0
:109AC00040D2DFE800F003080C11151A214D2D6873
:109AD000234E356037E0234D214E356033E04FF49F
:109AE00000451F4E35602EE0194D1D4E35602AE0B1
:109AF0004FF400451A4E356025E0184DDA352D68D3
:109B0000C5F30722154D263DD5F800512B0F134DF7
:109B1000DA352D6805F00304104D263DD5F80051C7
:109B200005F080050DB90A4901E00A4D2968651C58
:109B3000B1FBF5F5561C75435E1CB5FBF6F5084EFA
:109B4000356000E000BF00BF70BD0000840601402A
:109B50000024F400942B0020002D31012640054004
:109B6000902B002000127A0000B50748006840F4EE
:109B7000700005490860FFF791FF4FF4004002496B
:109B80008039086000BD000088ED00E002461068E2
:109B9000084008B1012070470020FCE72DE9F0479C
:109BA00081460D4617469A466FF0020875B36FB3AB
:109BB000D9F80C0000F4805616B1B6F5805F25D1B7
:109BC000002416E0534601228021484600F021F887
:109BD0008046B8F1000F00D00DE026B9295D484657
:109BE00000F033F804E035F81410484600F02DF882
:109BF000641CBC42E6D300BFB8F1000F06D1534647
:109C000001224021484600F004F880464046BDE865
:109C1000F087F8B505460E46144600270020009050
:109C20000AE00098984204D9581C10B16FF0070759
:109C300008E00098401C009031462846FFF7A6FF38
:109C4000A042EED100BF3846F8BD021D118070471A
:109C50000FB4054B10B503A9044A029800F04CF864
:109C600010BC5DF814FB000039A90000F882FF1F4A
:109C7000002807DB00F01F0201219140024A43093E
:109C800042F823107047000080E200E000280DDB5E
:109C900000BF00BF00F01F02012191404209920065
:109CA00002F1E022C2F8001100BF00BF70470000BF
:109CB00010B5002804DB0A07130E054A135406E00A
:109CC0000A07140E034A00F00F031B1FD45410BDE3
:109CD00000E400E018ED00E002E008C8121F08C12F
:109CE000002AFAD170477047002001E001C1121F1D
:109CF000002AFBD1704700002DE9FF4F8DB00F46C1
:109D00000546002606E025280BD0DDE90F12904716
:109D10006D1C761C28780028F5D111B03046BDE8BE
:109D2000F08F0024A246A1460122EC4900E0044342
:109D300015F8013F203B02FA03F00842F7D12878DA
:109D40002A2810D06FF02F022878A0F130010929BD
:109D500014D80AEB8A0102EB410144F0020400EB43
:109D6000010A6D1CF0E701CF5FEA000A03D544F455
:109D70000054CAF1000A44F002046D1C28782E2811
:109D800017D115F8010F44F004042A280ED06FF003
:109D90002F022878A0F1300109290AD809EB89019E
:109DA00002EB410100EB01096D1CF2E757F8049B3F
:109DB0006D1C28786C280FD006DC4C2817D068283A
:109DC0000DD06A2814D104E0742810D07A280FD15D
:109DD0000DE044F400140AE044F4801401E044F47B
:109DE00040146978814202D104F580146D1C6D1C09
:109DF0002A786E2A1FD00CDC632A31D004DC002ABA
:109E00008BD0582A11D1A3E0642A68D0692A0CD1DA
:109E100065E0732A2ED004DC6F2A73D0702A04D137
:109E20009BE0752A6FD0782A6ED01046DDE90F12BC
:109E30009047761C50E1C4F30250022806D0032854
:109E400009D0042801CF09D0066045E101CFF11700
:109E5000C0E9006140E101CF06803DE106703BE1D1
:109E600017F8040B8DF8000000208DF80100EB4678
:109E7000012003E057F804BB4FF0FF3061074FF0BB
:109E8000000102D40DE008F10101884649450FDACE
:109E90008045F8DB1BF808100029F4D108E008F130
:109EA000010188468142FADB1BF808100029F6D12F
:109EB000DDE90F23AAEB08008146214600F036F9C0
:109EC000304400EB080604E0DDE90F121BF8010B3B
:109ED0009047B8F10108F7D221464846F7E00A2139
:109EE000C4F302534FF0000B0891022B04D001CFB2
:109EF000C117032B09D00AE0FF1D27F00707F7E879
:109F0000020108E032E01FE020E000B2C117042B9C
:109F100001D140B2C117031E71F1000307DA4FF0FF
:109F2000000CD0EB0C006CEB01012D2302E02305AB
:109F300004D52B238DF82430012303E0E30701D05F
:109F40002023F7E7984658E00A2110E010210EE0A0
:109F500010204FF0000B08900CE010214FF0000B88
:109F600044F004044FF00809089103E008214FF081
:109F7000000B0891C4F30253022B04D001CF00213F
:109F8000032B06D006E0FF1D27F00707F7E80201C4
:109F900003E080B2042B00D1C0B24FF000082307C9
:109FA0002BD5702A07D0DDF820C08CF0100C5CEAAD
:109FB0000B0C05D00EE040238DF82430012308E07F
:109FC00050EA010306D030238DF824308DF8252087
:109FD00002239846DDF820C08CF0080C5CEA0B0CDC
:109FE0000BD150EA010301D1630706D530238DF868
:109FF00024304FF00108A9F10109582A04D038A2F1
:10A000000B9208AA0A920BE03AA2F9E75B46089A7B
:10A01000FEF79AF90B9B9B5C0A9A521E0A921370E8
:10A0200050EA0102F2D10A98ADEB000000F1200BDA
:10A03000600702D524F4803401E04FF00109D945CE
:10A0400002DDA9EB0B0000E0002000EB0B01414416
:10A050000890AAEB010AE00306D4DDE90F232146AC
:10A06000504600F063F806444FF0000908E009A9E3
:10A0700011F80900DDE90F12904709F10109761C7A
:10A08000C145F4DBE0030CD5DDE90F232146504642
:10A0900000F04CF8064404E0DDE90F123020904750
:10A0A000761C0899481E08900029F5DC08E00A98FB
:10A0B0000A990078491C0A91DDE90F129047761C35
:10A0C000BBF10001ABF1010BF1DC21465046DDE9AB
:10A0D0000F2300F019F806446D1C1BE60928010047
:10A0E000303132333435363738396162636465660E
:10A0F00000000000303132333435363738394142D0
:10A1000043444546000000002DE9F0410446002587
:10A110001E461746880404D405E039462020B0477F
:10A120006D1C641EF9D52846BDE8F0812DE9F0418B
:10A13000044600251E469046C80301D5302700E09E
:10A140002027880404D505E041463846B0476D1CF9
:10A15000641EF9D52846BDE8F08130B502460B46AD
:10A16000002400214FF6FF7010E0555C6840491C48
:10A17000002409E000F0010525B14AF2010585EA55
:10A18000600000E04010641C082CF3DB9942ECDB1B
:10A1900030BD000070B503460C460020002100BF12
:10A1A00008E05D5C4540EDB2054E36F8155085EA95
:10A1B0002020491CA142F4D3C543ADB2156070BD47
:10A1C0000080FF1F2DE9FF4FC7B0814615461C4692
:10A1D00000204690804620605A20DA4908701020FE
:10A1E00008712020C870489881B246AA4846FEF7F8
:10A1F00099FC8046B8F1000F03D100204BB0BDE8B8
:10A20000F08FBDF818014844CF4908602068C01D90
:10A21000206009F10700BDF818114618A8F10900DF
:10A2200080B24590C84800684079502802D0602824
:10A230007DD149E05020C3494871C3480068807906
:10A24000012804D0022814D0032838D123E00120AB
:10A25000BC4988713C20BD49887401200870216880
:10A2600048191922B949FEF7AFF820681930206063
:10A2700028E00220B34988710120B5490870022006
:10A280004870216848191422B149FEF79DF82068EA
:10A290001430206016E00320AA49887140F2DB40A8
:10A2A000AC4908803620A1F82F0021684819B12256
:10A2B000A849FEF789F82068B130206002E000204C
:10A2C00020609BE700BF1DE160209E4948719E48C9
:10A2D00000688079012806D002280FD0032816D004
:10A2E000042877D1FEE0002020609B48316801609F
:10A2F000716841603189018100207FE70020206082
:10A30000964831880180B1788170002076E703207B
:10A310008C498871924806600068B0F80100914944
:10A320000860002044904FF4807104A800E0E6E04B
:10A33000FEF763F84598401F87B289480068B0F877
:10A3400001004490864800680078012849D1864879
:10A3500001884498814244D100218448FFF765F97F
:10A360003A46F11C8248FEF72FF801230F22002104
:10A37000402000F012FE7F49096801F508303A4696
:10A380007B4900F0EFFA00230F221946402000F02D
:10A3900004FE7849096801F508303A4604A900F03E
:10A3A000D7FA394604A8FFF7D8FE0390F81C315CB1
:10A3B000381D305C01EB0021039881420BD16D48C0
:10A3C000006838446B49086067480088401C66494B
:10A3D000088001E090E000BF01216448FFF725F903
:10A3E00054E05F4800680078F0BB5F4801884498FB
:10A3F00081424BD1F078317900EB012080B203909B
:10A400007079B17900EB0120029001AA4FF4083075
:10A410000299FFF7BFFE0C2257494FF4703000F04D
:10A4200097FA48F6A540544908804FF400408860E8
:10A430000020888001990398884203D101204E4969
:10A44000488002E000214C4841800C224A494FF4E8
:10A45000703000F087FA0C2247494FF4703000F05A
:10A4600077FA72B600BF00E010E0BFF34F8F4348A9
:10A47000006800F4E06042490843001D3F4908605D
:10A48000BFF34F8F00BF00BF00BFFDE73648017824
:10A490002268501C2060A95433480088010A2268B1
:10A4A000501C2060A9542088801C2649A1F8010076
:10A4B0000846016829608188A9808079A8712846AA
:10A4C0002168FFF74AFE83462268501C206005F889
:10A4D00002B04FEA1B212268501C2060A95408F0EA
:10A4E000FF008BE60020206040F21722314625480D
:10A4F000FDF76AFF002081E6002020607EE6002054
:10A5000020607BE600BF2088801C0E49A1F8010076
:10A510000846016829608188A9808079A871284649
:10A520002168FFF71AFE82462268501C206005F859
:10A5300002A04FEA1A212268501C2060A95408F09A
:10A54000FF005BE60C82FF1F1482FF1F9028002093
:10A55000A9280020BD2800206E290020F482FF1FBA
:10A560001882FF1F1C82FF1F2082FF1F0000024075
:10A57000DC87FF1F2482FF1FD087FF1F0CED00E048
:10A580000000FA05782900200146AEE000BF00BFB8
:10A5900000BF00BF00BF00BF00BF00BF00BF00BFC3
:10A5A00000BF00BF00BF00BF00BF00BF00BF00BFB3
:10A5B00000BF00BF00BF00BF00BF00BF00BF00BFA3
:10A5C00000BF00BF00BF00BF00BF00BF00BF00BF93
:10A5D00000BF00BF00BF00BF00BF00BF00BF00BF83
:10A5E00000BF00BF00BF00BF00BF00BF00BF00BF73
:10A5F00000BF00BF00BF00BF00BF00BF00BF00BF63
:10A6000000BF00BF00BF00BF00BF00BF00BF00BF52
:10A6100000BF00BF00BF00BF00BF00BF00BF00BF42
:10A6200000BF00BF00BF00BF00BF00BF00BF00BF32
:10A6300000BF00BF00BF00BF00BF00BF00BF00BF22
:10A6400000BF00BF00BF00BF00BF00BF00BF00BF12
:10A6500000BF00BF00BF00BF00BF00BF00BF00BF02
:10A6600000BF00BF00BF00BF00BF00BF00BF00BFF2
:10A6700000BF00BF00BF00BF00BF00BF00BF00BFE2
:10A6800000BF00BF00BF00BF00BF00BF00BF00BFD2
:10A6900000BF00BF00BF00BF00BF00BF00BF00BFC2
:10A6A00000BF00BF00BF00BF00BF00BF00BF00BFB2
:10A6B00000BF00BF00BF00BF00BF00BF00BF00BFA2
:10A6C00000BF00BF00BF00BF00BF00BF00BF00BF92
:10A6D00000BF00BF00BF00BF00BF00BF00BF00BF82
:10A6E00000BF00BF00BF4A1E91B200293FF74EAF26
:10A6F00070470146B5E000BF00BF00BF00BF00BF0C
:10A7000000BF00BF00BF00BF00BF00BF00BF00BF51
:10A7100000BF00BF00BF00BF00BF00BF00BF00BF41
:10A7200000BF00BF00BF00BF00BF00BF00BF00BF31
:10A7300000BF00BF00BF00BF00BF00BF00BF00BF21
:10A7400000BF00BF00BF00BF00BF00BF00BF00BF11
:10A7500000BF00BF00BF00BF00BF00BF00BF00BF01
:10A7600000BF00BF00BF00BF00BF00BF00BF00BFF1
:10A7700000BF00BF00BF00BF00BF00BF00BF00BFE1
:10A7800000BF00BF00BF00BF00BF00BF00BF00BFD1
:10A7900000BF00BF00BF00BF00BF00BF00BF00BFC1
:10A7A00000BF00BF00BF00BF00BF00BF00BF00BFB1
:10A7B00000BF00BF00BF00BF00BF00BF00BF00BFA1
:10A7C00000BF00BF00BF00BF00BF00BF00BF00BF91
:10A7D00000BF00BF00BF00BF00BF00BF00BF00BF81
:10A7E00000BF00BF00BF00BF00BF00BF00BF00BF71
:10A7F00000BF00BF00BF00BF00BF00BF00BF00BF61
:10A8000000BF00BF00BF00BF00BF00BF00BF00BF50
:10A8100000BF00BF00BF00BF00BF00BF00BF00BF40
:10A8200000BF00BF00BF00BF00BF00BF00BF00BF30
:10A8300000BF00BF00BF00BF00BF00BF00BF00BF20
:10A8400000BF00BF00BF00BF00BF00BF00BF00BF10
:10A8500000BF00BF00BF00BF00BF00BF00BF4A1E57
:10A8600091B200293FF747AF704700000121012056
:10A870000B4A12680AB1002011E00A4A12680AB1B4
:10A8800000200CE0084A12680AB1002007E0074ADD
:10A890001368074A1268521E934200D10220704783
:10A8A0002CB0FF1F8C82FF1F8882FF1F54B0FF1F38
:10A8B0007882FF1F08B503220021012002F010FA60
:10A8C000174908600020009028E04FF0FF3114483D
:10A8D000006802F083FC00201249087012480088CA
:10A8E00010B94FF4807000E000200F49088000206C
:10A8F000088000900D48098842186B464FF400719B
:10A900000B48FFF75FFC012006490870009808B16A
:10A91000002001E045F2665006490880D5E70000B6
:10A920005C82FF1F6082FF1F5282FF1FF1A8FF1F82
:10A93000F1AAFF1F5082FF1F13B50C46FF2301220F
:10A9400069460248FFF72AF900981CBD00D0014073
:10A9500070B504460D461646324629462046FDF798
:10A960006BFF70BD2DE9F74F074614464FEA573984
:10A97000BB464FEA5B35CBF30C0ACAF50056B4422E
:10A9800000D82646C720FEF795FA0120FDF7A8FE5D
:10A9900058E0002101EB45304FF400522E49FFF7FB
:10A9A000D7FF4FF0000807E02B4810F80800FF28F9
:10A9B00000D004E008F10108B8F5005FF4D300BF4F
:10A9C000B0451ED209F0FF000121FDF7DFFF002195
:10A9D00001EB4530FDF762FF1F4901EB0A003246EB
:10A9E0000199FDF7F1FC002101EB45304FF40052D5
:10A9F0001949FDF797FE09F0FF000021FDF7C6FF9A
:10AA00000EE009F0FF000121FDF7C0FF3246384695
:10AA10000199FDF787FE09F0FF000021FDF7B6FF61
:10AA2000B44200D10FE06D1C4FF0000A0198304491
:10AA300001903744A41BB4F5005F02D94FF40056CF
:10AA400000E02646A5E700BF0020FDF749FEC7202D
:10AA5000FEF778FABDE8FE8FDC88FF1F00B587B0EF
:10AA600001A8FEF75DF90220ADF806000020ADF860
:10AA7000040001AA4FF480610220FEF7ADF801AA9C
:10AA80004FF400610220FEF7A7F84FF48061022026
:10AA9000FEF72CF94FF400610220FEF727F907B00A
:10AAA00000BD00B587B001A8FEF73AF90220ADF865
:10AAB00006000020ADF8040001AA4FF40061FEF783
:10AAC0008BF801AA4FF480510020FEF785F84FF46F
:10AAD00000610020FEF70AF94FF480510020FEF7D4
:10AAE00005F907B000BD70B506460024FEF766FD07
:10AAF00000251BE04FF400610220FEF7D5F8052089
:10AB0000FFF742FD4FF400610220FEF7EFF8600608
:10AB1000040E4FF480610220FEF7B8F808B1601C03
:10AB2000C4B20520FFF730FD681CC5B2082DE1DB7B
:10AB3000204670BD70B506460024FEF74CFD01208E
:10AB4000FFF7D7FD00251BE04FF400610020FEF762
:10AB5000ABF80520FFF7CDFD4FF400610020FEF7B4
:10AB6000C5F86006040E4FF480510020FEF78EF801
:10AB700008B1601CC4B20520FFF7BBFD681CC5B25C
:10AB8000082DE1DB204670BD70B50446FEF72FFDB1
:10AB90004FF400610220FEF787F8002521E004F061
:10ABA000800028B14FF480610220FEF79FF804E096
:10ABB0004FF480610220FEF777F86006040E05204E
:10ABC000FFF7E2FC4FF400610220FEF78FF805204A
:10ABD000FFF7DAFC4FF400610220FEF765F8681C0D
:10ABE000C5B2082DDBDB70BD70B50446FEF70EFD67
:10ABF0004FF400610020FEF757F8002521E004F033
:10AC0000800028B14FF480510020FEF76FF804E077
:10AC10004FF480510020FEF747F86006040E05202F
:10AC2000FFF767FD4FF400610020FEF75FF8052095
:10AC3000FFF75FFD4FF400610020FEF735F8681C58
:10AC4000C5B2082DDBDB70BD10B5FEF7D0FC4FF4AC
:10AC500080610220FEF74AF84FF400610220FEF7FF
:10AC600045F80520FFF790FC4FF480610220FEF7C5
:10AC70001BF80520FFF788FC4FF400610220FEF767
:10AC800013F810BD10B5FEF7C1FC4FF48051002041
:10AC9000FEF72CF84FF400610020FEF727F805209E
:10ACA000FFF727FD4FF480510020FDF7FDFF052041
:10ACB000FFF71FFD4FF400610020FDF7F5FF10BD09
:10ACC00010B5FEF794FC4FF400610220FDF7ECFF95
:10ACD0004FF480610220FDF7E7FF0520FFF754FCE9
:10ACE0004FF400610220FEF701F84FF4806102206A
:10ACF000FDF7FCFF0520FFF747FC10BD10B5FEF780
:10AD000085FC4FF400610020FDF7CEFF4FF4805129
:10AD10000020FDF7C9FF0520FFF7EBFC4FF40061B1
:10AD20000020FDF7E3FF4FF480510020FDF7DEFF28
:10AD30000520FFF7DEFC10BD10B5C824FEF757FC58
:10AD40004FF480610220FDF7D1FF0120FFF71CFCCA
:10AD50004FF400610220FDF7C9FF0120FFF714FC4A
:10AD6000FEF72CFC09E0601E84B21CB9FFF7A8FFB7
:10AD7000012010BD0120FFF707FC4FF48061022085
:10AD8000FDF784FF0028EED14FF400610220FDF7AB
:10AD90008BFF0020EDE710B5C824FEF737FC4FF419
:10ADA00080510020FDF7A2FF0120FFF7A2FC4FF425
:10ADB00000610020FDF79AFF0120FFF79AFCFEF7E3
:10ADC0000AFC09E0601E84B21CB9FFF797FF01205E
:10ADD00010BD0120FFF78DFC4FF480510020FDF7DE
:10ADE00055FF0028EED14FF40061FDF75DFF002014
:10ADF000EEE700001CB5C720FEF75CF801F044FA4E
:10AE000000F0E2FF00F06EF800F09CF801F061F84D
:10AE1000C720FEF797F80020022103460A02CDE979
:10AE200000101DA1204802F0FDFA00200321034676
:10AE30004FF40072CDE900101CA11F4802F0F2FA95
:10AE400000201F2103464FF40072CDE900101BA122
:10AE50001D4802F0E7FA0020032103464FF4007278
:10AE6000CDE9001019A11C4802F0DCFA01F0C8FD80
:10AE700011E000BFBFF34F8F1848006800F4E06096
:10AE800017490843001D15490860BFF34F8F00BFE5
:10AE900000BF00BFFDE7ECE76E6361393535355F14
:10AEA0007461736B0000000085B00000737936395F
:10AEB00037305F7461736B00BDC00000656336306E
:10AEC00030675F7461736B00B5A800006D70755FCB
:10AED0007461736B0000000015AF00000CED00E022
:10AEE0000000FA0500B587B001A8FDF719FF0220A0
:10AEF000ADF806000020ADF8040001AA04210520E9
:10AF0000FDF76AFE01AA4FF440410220FDF764FEFE
:10AF100007B000BD04210520FDF7E8FE4FF4804195
:10AF20000220FDF7E3FE4FF47A7001F04FFC4FF47E
:10AF300080410220FDF7B8FE03E04FF4FA7001F003
:10AF400045FCFAE710B5FFF789FD10BD2DE9F0418A
:10AF500007460C4615461E464FF00008FFF774FEE4
:10AF60003846FFF711FEFFF7E7FE80462846FFF759
:10AF70000BFEFFF7E1FE8046FFF766FE2046FFF777
:10AF800003FEFFF7D9FE80460020FFF7ACFD3070CE
:10AF9000FFF796FE0020BDE8F081F8B504460E46A6
:10AFA00015461F4600200090012E01DC802D00DD9B
:10AFB000F8BDD6B944F001016B4602222046FFF7E6
:10AFC000C5FF012F08D19DF8001041EA0502204677
:10AFD000022100F06FF824E09DF8001021EA05023C
:10AFE0002046022100F066F81BE0012E19D144F042
:10AFF00001016B4603222046FFF7A8FF012F08D16D
:10B000009DF8001041EA05022046032100F052F8A5
:10B0100007E09DF8001021EA05022046032100F018
:10B0200049F800BFC4E7F8B504460D4616460020AF
:10B030000090012D01DC802E00DDF8BD7DB944F0CB
:10B0400001016B4606222046FFF780FF9DF80010A5
:10B0500021EA06022046062100F02CF810E0012D1E
:10B060000ED144F001016B4607222046FFF76EFF28
:10B070009DF8001021EA06022046072100F01AF888
:10B0800000BFDAE7C0B00F2200214020FFF7CBFF5E
:10B090004FF4807206496846FDF796F907E04FF4D1
:10B0A000FA7001F093FB44F2506001F08FFBF6E779
:10B0B00038DB00002DE9F04106460C461546012715
:10B0C000FFF7C2FD3046FFF75FFDFFF735FE07468D
:10B0D0002046FFF759FDFFF72FFE07462846FFF7EA
:10B0E00053FDFFF729FE0746FFF7EAFD0020BDE804
:10B0F000F08100002DE9F04105460E46264807681C
:10B1000026480068001D01F01DF950B92348006869
:10B1100090F82C100120884021490968814320487B
:10B120000160681CD8B9D6B11E4948681B49096836
:10B1300088601A4982680968CA6018490968091D47
:10B140008268516015490968091D8160154A1349D3
:10B1500009684A6111460968491C11601AE07C19A6
:10B160000E4800684460BC4207D20C480168091DC3
:10B170000D48006801F00AF90CE008480168091D53
:10B180000A48006801F002F909480068844201D2C7
:10B1900007480460BDE8F0817C82FF1F6882FF1FC2
:10B1A0008082FF1F54B0FF1F7082FF1F6C82FF1F41
:10B1B0009882FF1F10B5044601F002F9314800687B
:10B1C000401C304908603048006840B92E4804608F
:10B1D0000846006801280DD100F05EFA0AE02B480D
:10B1E000006838B928480068C06AE16A884201D816
:10B1F0002548046026480068401C25490860084628
:10B200000068606494F82C10012088402149096886
:10B21000084320490860E16A01EB81011E4A02EB04
:10B2200081014868A0608268E260211D82685160E7
:10B230008160E16A01EB8101174A02EB81026261E0
:10B24000E16A01EB8101144A52F82110491CE26ABB
:10B2500002EB8202104B43F8221001F0DBF80B489E
:10B26000006868B108480068C06AE16A884207D28D
:10B270004FF0805009490860BFF34F8FBFF36F8FC5
:10B2800010BD00007882FF1F6882FF1F8482FF1FAD
:10B290009482FF1F8082FF1F84ADFF1F04ED00E03A
:10B2A00010B501F08DF810480068D0B90F4801F0D2
:10B2B0005DF80F4801F05AF80C480E4908600C4838
:10B2C0000D49086000220C210A2001F009FD064901
:10B2D00008600846006820B108A10348006801F032
:10B2E0001FFA01F097F810BDB082FF1F68B0FF1F72
:10B2F0007CB0FF1FA882FF1FAC82FF1F546D7251EC
:10B300000000000010B516E001F05AF80C48C068C3
:10B31000C468201D01F016F80A480068401E09495B
:10B32000086009480068401E0749086001F072F88B
:10B33000204600F05FF8044800680028E4D110BD02
:10B3400040B0FF1F7882FF1F7482FF1F70B5044654
:10B350000D46206C70B1216CE0680144E160D4E9D5
:10B360000210884201D32168E1602846226CE1681E
:10B37000FDF72AF870BD2DE9F04104460F46154649
:10B380004FF00008A66B206C48B9206800282CD12B
:10B39000A06802F06BF980460020A06025E07DB92E
:10B3A0003946226C6068FDF70FF8216C606808442C
:10B3B0006060D4E90101884217D32068606014E01E
:10B3C0003946226CE068FCF7FFFF216CE068411A07
:10B3D000E1602168E068884203D2216CA068411ACC
:10B3E000E160022D01D106B1761E701CA0634046BB
:10B3F000BDE8F08110B50446206B01F029F8204625
:10B4000001F026F810BD01464A6A22B10A6B1268A3
:10B41000C2F1200000E0002070470000002101225E
:10B420000C4B1B68012B00D901210B4A1268D26A10
:10B430000AB100200DE0094A1268012A01D9002052
:10B4400007E009B1002004E0054A1268054B1B68BB
:10B45000D01A70478082FF1F6882FF1F84ADFF1FD4
:10B460009882FF1F7C82FF1F0146084A12681268FB
:10B470000AB9012200E000220A600A6822B9034AE0
:10B480001268D268106800E000207047A882FF1F91
:10B4900030B54FF4F043174800F007042CB1C01D3D
:10B4A00020F00700134C041B1B1B0246124C2260A9
:10B4B0000024114D6C60D018083820F007000F4CA4
:10B4C000206000240D4D2D686C600C4D2D682C60A3
:10B4D0001146441A4C60094C24680C60084D4C68B5
:10B4E0002C60084D4C682C604FF00044064D2C60D9
:10B4F00030BD000090B0FF1FBC82FF1FC482FF1F41
:10B50000CC82FF1FC882FF1FD882FF1F00BFFFF73A
:10B51000F9FE19480068012807D94FF080501749F3
:10B520000860BFF34F8FBFF36F8FFFF777FF0446BD
:10B53000022C20D301F0D2FA1148006811490968A1
:10B54000884201D3012000E0002050B900BF502004
:10B5500080F31188BFF34F8FBFF36F8F00BF00BF21
:10B56000FEE7FFF75BFF0446022C02D3204600F003
:10B57000F5FF02F0FBF9CAE784ADFF1F04ED00E020
:10B580009882FF1F7C82FF1F2DE9F04106460D4681
:10B5900017469846069C0DB9246000E02760E663D4
:10B5A00025640121204601F0CFFB84F85080002063
:10B5B000A064BDE8F0812DE9F05F82460F46904619
:10B5C0009B460A9E0C9C4FEA8801A522206BFCF743
:10B5D0000DFFA8F10100216B01EB800929F007099B
:10B5E00009F0070008B9012000E0002050B900BFB1
:10B5F000502080F31188BFF34F8FBFF36F8F00BFD0
:10B6000000BFFEE787B1002507E0795D04F1340053
:10B610004155785D00B902E06D1C102DF5D300BFD7
:10B6200000214320015502E0002084F83400202E40
:10B6300001D2012000E0002050B900BF502080F36B
:10B640001188BFF34F8FBFF36F8F00BF00BFFEE7BE
:10B65000202E00D31F26E662E66400202065201D10
:10B6600000F091FE04F1180000F08DFE2461C6F197
:10B670002000A06164620020606584F858005A468A
:10B680005146484600F08AFB20600B9808B10B98A1
:10B690000460BDE8F09F000010B5002407E004EB53
:10B6A00084010F4A02EB810000F060FE641C202C34
:10B6B000F5D30C4800F05AFE0B4800F057FE0B483B
:10B6C00000F054FE0A4800F051FE0A4800F04EFE19
:10B6D00004480949086004480849086010BD000092
:10B6E00084ADFF1F04B0FF1F18B0FF1F2CB0FF1F59
:10B6F00040B0FF1F54B0FF1F6C82FF1F7082FF1FFE
:10B7000010B50146164800E0006803688B42FBD381
:10B710000246436813448B4204D143684C68234477
:10B72000436001460A464B6813440468A34211D1A2
:10B730000C4C03682468A34208D04B680468646812
:10B7400023444B6003681B680B6005E0054B1B68D6
:10B750000B6001E003680B60884200D0016010BDFF
:10B76000BC82FF1FC482FF1F2DE9F04104460D4635
:10B7700016461F464FF0000865602461B5420CD89C
:10B78000F01BA169884202D34FF0010811E0211D8E
:10B790000948006800F0FAFD0BE0BE4204D2BD4249
:10B7A00002D34FF0010804E0211D0448006800F0B6
:10B7B000EDFD4046BDE8F081AC82FF1FA882FF1F6F
:10B7C00070B5054600F0FCFDA86B08B9012400E047
:10B7D000002400F01FFE204670BDF1B50098846C77
:10B7E000002654B900BF502080F31188BFF34F8F5B
:10B7F000BFF36F8F00BF00BFFEE7A06BE16B884215
:10B8000001D2012000E0002050B900BF502080F399
:10B810001188BFF34F8FBFF36F8F00BF00BFFEE7EC
:10B82000A06BE16B88422CD294F945500022694606
:10B830002046FFF7A0FD0646681C60B9606A08B99B
:10B84000012000E00020D8B904F1240001F0FCFF41
:10B85000B0B1012614E07F2D01D0012000E00020CE
:10B8600050B900BF502080F31188BFF34F8FBFF352
:10B870006F8F00BF00BFFEE7681C40B284F8450030
:10B8800000BF3046F8BD000070B505460E460E48B4
:10B890000068C068C468201D00F054FD94F82800BA
:10B8A00000F0040028B132462946204600F0D6F8C0
:10B8B00005E094F8280000F0FE0084F828002046F7
:10B8C000216A884770BD0000A882FF1F7FB57FE016
:10B8D000019800287CDB039C606908B9012000E026
:10B8E000002010B9201D00F02DFD684600F0E2F8A0
:10B8F000054601980A2869D2DFE800F06805072E9E
:10B90000365806082F3700BF00BF00BF94F8280044
:10B9100040F0010084F828000298A26981180346CB
:10B920002A462046FFF720FFA8B194F8280000F02F
:10B93000040038B10298A26981182A46204600F016
:10B940008DF805E094F8280000F0FE0084F8280047
:10B950002046216A88473AE000BF94F8280000F0AA
:10B96000FE0084F8280032E000BF94F8280040F080
:10B97000010084F828000298A061A06908B10120A4
:10B9800000E0002050B900BF502080F31188BFF3C1
:10B990004F8FBFF36F8F00BF00BFFEE7A069411953
:10B9A0002B462A462046FFF7DFFE10E094F82800D9
:10B9B00000F0020018B9204600F04AFD05E094F8B6
:10B9C000280000F0FE0084F8280000E000BF00BF5F
:10B9D000002201A90348006801F04CFB00287FF415
:10B9E00077AF7FBDB082FF1FF8B505460C4601F06A
:10B9F00075F8684600F05EF80646009820BB44B92A
:10BA0000B54206D801F0B2FF31462846FFF73CFFA9
:10BA10001CE03CB10E480068006808B9012000E055
:10BA200000200446A91B22460A48006800F0A8FE30
:10BA300001F09CFF50B94FF0805007490860BFF3F8
:10BA40004F8FBFF36F8F01E001F090FFF8BD000052
:10BA5000AC82FF1FB082FF1F04ED00E070B504460A
:10BA60000D46164604E0A06905442046216A884731
:10BA7000A06941192B4632462046FFF775FE002883
:10BA8000F1D170BD09480068006808B9012000E0E4
:10BA9000002020B14FF0FF300549086005E0034861
:10BAA0000068C06800680249086070476C82FF1F28
:10BAB0009882FF1F70B5044601F0F4FC0546074864
:10BAC0000068854204D200F00BF80120206001E0FC
:10BAD0000020206001480560284670BDB882FF1F25
:10BAE00070B508E00D480068C06804684FF0FF3189
:10BAF0002046FFF7C9FE09480068006808B9012020
:10BB000000E000200028EDD00448056804480068E3
:10BB1000024908600248056070BD0000A882FF1F4E
:10BB2000AC82FF1F0E480068401C08B9012000E0ED
:10BB3000002050B900BF502080F31188BFF34F8F11
:10BB4000BFF36F8F00BF00BFFEE700BF502080F340
:10BB50001188BFF34F8FBFF36F8F00BF00BFFEE7A9
:10BB6000DC82FF1F08B500BF6846FFF77DFC044676
:10BB700020460099FFF738FFFFF7A8FEF4E770B5FD
:10BB8000044600F01DFC94F9455019E0A06C30B15A
:10BB90002046FFF722FE88B100F052FE0EE0606AF8
:10BBA00008B9012000E0002038B904F1240001F0B8
:10BBB0004BFE18B100F044FE00E003E0681E45B201
:10BBC000002DE3DC00BFFF2084F8450000F022FCDC
:10BBD00000F0F6FB94F9445010E0206908B9012008
:10BBE00000E0002048B904F1100001F02DFE08B17A
:10BBF00000F026FE681E45B200E001E0002DECDCFE
:10BC000000BFFF2084F8440000F004FC70BD000079
:10BC10002DE9F04104464FF0000800F05FFF514865
:10BC2000006808B9FFF734FC4F480068204000283E
:10BC30007ED13CB304F10800A04223D9083404F0BB
:10BC4000070000B304F00700C0F108002044A04240
:10BC500016D904F00700C0F10800044404F00700FE
:10BC600008B9012000E0002068B900BF502080F32F
:10BC70001188BFF34F8FBFF36F8F00BF00BFFEE788
:10BC8000002400E00024002C54D03848006884428E
:10BC900050D8374E3046056801E02E462D6868685A
:10BCA000A04202D228680028F7D12E4800688542B9
:10BCB00040D0306800F10808286830606868001BD0
:10BCC000102819D92F1907F0070008B9012000E042
:10BCD000002050B900BF502080F31188BFF34F8F70
:10BCE000BFF36F8F00BF00BFFEE76868001B78607E
:10BCF0006C603846FFF704FD1C4968680968081A3B
:10BD00001A490860084600681A490968884203D23F
:10BD100016480068174908601349686809680843AD
:10BD200068600020286014480068401C124900E048
:10BD300000E0086001F01AFE08F0070008B90120D1
:10BD400000E0002050B900BF502080F31188BFF3FD
:10BD50004F8FBFF36F8F00BF00BFFEE74046BDE8C7
:10BD6000F0810000C482FF1FD882FF1FC882FF1F1E
:10BD7000BC82FF1FCC82FF1FD082FF1F06480068D5
:10BD800030B10549096801F15000096D491C016095
:10BD900001480068704700006882FF1F001F4FF0D5
:10BDA00080730360001F21F001030360001F054B37
:10BDB000036014380260001F6FF002030360203834
:10BDC0007047000025BB000000B58DB02B228021FC
:10BDD0000120FCF775FF28224FF400710120FCF7C9
:10BDE0006FFF29224FF480710120FCF769FF0121C8
:10BDF0008804FCF787FE02A8FDF700FD01200290F1
:10BE000000200390049006900320079049F204005C
:10BE100008904FF48060099000200A900C9002A9CD
:10BE20002248FDF70EFC012291022048FDF745FC57
:10BE3000012251021D48FDF740FC40F27310ADF89D
:10BE400000000720ADF80200194801906846FCF791
:10BE50007BFFBDF90200FDF70BFFBDF902000E21CB
:10BE6000FDF726FFBDF90200FDF710FF4FF4BA7091
:10BE7000ADF800000820ADF802000E4801906846B9
:10BE8000FCF762FFBDF90200FDF7F2FEBDF902000A
:10BE90000E21FDF70DFFBDF90200FDF7F7FE0121B0
:10BEA0000248FDF7C2FB0DB000BD000000000240DB
:10BEB000D59600003198000038B504460020009067
:10BEC0006A462146D42000F008F89DF80010084684
:10BED00038BD10B5FEF7E5FD10BD70B504460D4642
:10BEE0001646FEF7CFFE2046FEF77EFEFEF753FF16
:10BEF0002846FEF779FEFEF74EFFFEF7C3FE44F03C
:10BF00000100FEF771FEFEF746FF0020FEF712FE6D
:10BF10003070FEF7F3FE70BD38B505460C460020C4
:10BF20000090072D7DD2DFE805F004BE1A4788BED9
:10BF300099009DF8000020F0800000909DF800001E
:10BF400020F0400040300090A4F16400322190FBCA
:10BF5000F1F09DF8001060F305010091A5E09DF857
:10BF6000000020F08000803000909DF8000020F05C
:10BF7000400000909DF8000020F0200000909DF807
:10BF8000000020F01000103000909DF8000020F01C
:10BF90000800083000909DF8000020F00400001D0B
:10BFA00000909DF8000020F0020000909DF8000035
:10BFB00020F00100009078E014B1012C39D11AE092
:10BFC0009DF8000020F0800000909DF8000020F017
:10BFD000400000909DF8000020F0200000909DF8A7
:10BFE000000020F0100000909DF8000020F00E00EE
:10BFF0000A3000901FE09DF8000020F080000090C3
:10C000009DF8000020F0400000909DF8000020F016
:10C01000200000909DF8000020F0100010300090EB
:10C0200000E040E09DF8000020F00E000A30009093
:10C0300001E0012038BD00BF37E02046E11704EBE6
:10C040009161C1F38F149DF8000020F080000090F2
:10C050009DF8000064F30600009026E040F6DC60E6
:10C06000844201DA0020E5E7A4F580517039002907
:10C0700006D4A4F57060C11700EB1171091100E03E
:10C0800017218CB29DF8000064F3820000909DF8A7
:10C09000000020F00200801C00909DF8000020F0BD
:10C0A0000100009001E00120C4E700BF9DF80020DE
:10C0B0002946D42000F0D0F80020BBE708B54FF4A3
:10C0C00080605949088041F27000584908804FF457
:10C0D0007A705749088000210220FFF71DFF54485D
:10C0E00001880020FFF718FF4F4801880420FFF760
:10C0F00013FF4E4801880620FFF70EFF92E00E2046
:10C10000FFF7DAFE00904B489DF8001001700078B0
:10C1100000F07F0000EB80004FF4106101EB800025
:10C12000454908800F20FFF7C7FE009041489DF861
:10C1300000100170007800F07F0000EB80004FF4E9
:10C14000106101EB80003D4908800B20FFF7B4FE31
:10C15000009038489DF8001001700078C0F3C100CD
:10C16000374908700C20FFF7A7FE009031489DF872
:10C1700000100170007800F00300324908701220AE
:10C18000FFF79AFE00902B489DF800100170007890
:10C1900000F07F00322110FB01F02B4908801320B2
:10C1A000FFF78AFE009023489DF800100170007888
:10C1B00000F03F00254908701F480088B0F5845FF3
:10C1C0000BDD23480078012807D100210320FFF769
:10C1D000A3FE00201E4908700EE017480088B0F545
:10C1E0007A6F09DA1A48007830B901210320FFF785
:10C1F00093FE01201649087000210220FFF78CFEF3
:10C200004FF47A7000F0E2FA002409E02046FFF7CC
:10C2100053FE00900F489DF800100155601CC4B2F9
:10C22000142CF3DD6BE700004882FF1F4682FF1FDE
:10C230004A82FF1F4282FF1F3C82FF1F3E82FF1F78
:10C240004082FF1F4382FF1F4C82FF1F4582FF1F5A
:10C250004E82FF1FDCA8FF1F70B506460C46154630
:10C26000FEF710FD3046FEF7BFFCFEF794FD2046BA
:10C27000FEF7BAFCFEF78FFD2846FEF7B5FCFEF789
:10C280008AFDFEF73BFD70BD0EB52C492C48FCF72E
:10C2900092F9012203210520FCF77EFC02A8FCF79D
:10C2A00009FA00208DF80A0030208DF809000020DE
:10C2B0008DF8080005208DF80B0002A8FCF7D8F9CE
:10C2C0006846FCF74FF900208DF8000001900198B6
:10C2D00020F0030001906321019861F31020019088
:10C2E000019820F0704000F1E0400190019820F0AA
:10C2F000706000F1E0600190019820F4700000F59A
:10C30000E0000190019820F0800001906846FCF761
:10C3100009F9002211460320FDF7ACFA012211466B
:10C320000420FDF7A7FA0320FCF708FB4FF4405068
:10C33000FCF7E8FC0520FCF748F90EBD10221100BF
:10C340007777770701460A69D1E901309860D1E92A
:10C35000010358605068884201D18868506000200D
:10C3600008611068401E10601068704700F10801F5
:10C3700041604FF0FF31816000F10801C16001614F
:10C3800000210160704700210161704710B502462D
:10C390000B685C1C0CB9106907E002F1080000E0B2
:10C3A0004068446824689C42FAD944684C604C68F0
:10C3B000A160886041600A611468641C146010BD4B
:10C3C00000BF502080F31188BFF34F8FBFF36F8FF2
:10C3D00000BF0E480068401C0C4908600846006811
:10C3E000012812D10A480068C0B208B9012000E053
:10C3F000002050B900BF502080F31188BFF34F8F49
:10C40000BFF36F8F00BF00BFFEE77047DC82FF1FE6
:10C4100004ED00E00D48006850B900BF502080F3E3
:10C420001188BFF34F8FBFF36F8F00BF00BFFEE7D0
:10C4300006480068401E054908600846006820B9A3
:10C44000002080F3118800BF00BF7047DC82FF1F0F
:10C4500070B506463546002E44D0083D2C4622498C
:10C4600060680968084008B1012000E0002050B968
:10C4700000BF502080F31188BFF34F8FBFF36F8F41
:10C4800000BF00BFFEE7206808B9012000E00020DF
:10C4900050B900BF502080F31188BFF34F8FBFF316
:10C4A0006F8F00BF00BFFEE70F4960680968084052
:10C4B000C0B12068B0B90C49606809688843606001
:10C4C00000F00CFB094960680968084407490860E6
:10C4D0002046FFF715F906480068401C044908602B
:10C4E00001F044FA70BD0000D882FF1FC882FF1F10
:10C4F000D482FF1F154800684FF47A71B0FBF1F049
:10C5000013490860084600686FF07F41B1FBF0F006
:10C51000104908600D480068B0FBF0F02D21B1FB18
:10C52000F0F00D49086000204FF0E02108618861BB
:10C53000064800684FF47A71B0FBF1F0401E4FF0EE
:10C54000E02148610720086170470000902B00201F
:10C55000E082FF1FE482FF1FE882FF1F2DE9F04108
:10C5600004464E480068844201D94C4804684FF0A4
:10C57000E020006920F001004FF0E021086108464A
:10C580008169601E464A126802FB00154548006832
:10C59000854202D9434800682D1A72B6BFF34F8F07
:10C5A000BFF36F8FFEF762F980B94FF0E02080692A
:10C5B0004FF0E02148610846006940F00100086141
:10C5C00037480068401E486162B665E04FF0E020E1
:10C5D000456100204FF0E02188610846006940F085
:10C5E00001000861A046B8F1000F04D0BFF34F8FDF
:10C5F00030BFBFF36F8F62B6BFF34F8FBFF36F8F44
:10C6000072B6BFF34F8FBFF36F8F06204FF0E0215C
:10C6100008610846006900F48030B8B12049096813
:10C62000491E4FF0E0229269AA1A881A1D4909682A
:10C63000884203D31A490968884202D9184909680F
:10C64000481E4FF0E0214861661E12E01448006861
:10C6500060434FF0E0218969471A11480068B7FB31
:10C66000F0F6701C0E4909684843C01B4FF0E021EA
:10C67000486100204FF0E02188610846006940F0E1
:10C6800001000861304600F009FA05480068401EC4
:10C690004FF0E021486162B6BDE8F081E482FF1FFF
:10C6A000E082FF1FE882FF1F70B5FBF737FE0446EC
:10C6B000102C16D304F1E02090F8F05315480078C0
:10C6C000854201DB012000E0002050B900BF50206E
:10C6D00080F31188BFF34F8FBFF36F8F00BF00BF90
:10C6E000FEE70D48006800F4E0600C4909688842E4
:10C6F00001D8012000E0002050B900BF502080F395
:10C700001188BFF34F8FBFF36F8F00BF00BFFEE7ED
:10C7100070BD0000EC82FF1F0CED00E0F082FF1FF7
:10C7200030B502460B4652B900BF502484F311883D
:10C73000BFF34F8FBFF36F8F00BF00BFFEE7002135
:10C74000BBB1002012E00D4C04EBC00464689442BD
:10C7500003D10A4C04EBC0010AE031B9074C54F88C
:10C76000304014B9054C04EBC001401C0A28EAD340
:10C7700000BF09B10B604A6030BD000034ADFF1F3F
:10C780002DE9F04105460E4617462C46FFF718FEE8
:10C7900094F94400401C10B9002084F8440094F936
:10C7A0004500401C10B9002084F84500FFF732FE18
:10C7B000A06B28B93A46314604F1240000F062F833
:10C7C0002046FFF7DCF9BDE8F081000070B50446B3
:10C7D0000025D4B11248006808B9012000E000200B
:10C7E00050B900BF502080F31188BFF34F8FBFF3C3
:10C7F0006F8F00BF00BFFEE700F070F900212046F8
:10C80000FEF778FC01F0B2F805463DB94FF08050D4
:10C8100004490860BFF34F8FBFF36F8F70BD0000F6
:10C82000A482FF1F04ED00E0034909680160034989
:10C8300009684160704700009082FF1F7C82FF1FE3
:10C8400001200149086070478C82FF1F70B50446C3
:10C850000D4654B900BF502080F31188BFF34F8FAD
:10C86000BFF36F8F00BF00BFFEE7054801681831B6
:10C870002046FFF78BFD01212846FEF73BFC70BDEB
:10C880006882FF1F70B504460E46154654B900BFB6
:10C89000502080F31188BFF34F8FBFF36F8F00BF1D
:10C8A00000BFFEE760680F490968C8610D498268EA
:10C8B00009680A620B4909681831826851600949A0
:10C8C000096818318160074909688C622168491C30
:10C8D00021600DB14FF0FF3629463046FEF70AFCC5
:10C8E00070BD00006882FF1F2DE9F04706460F4625
:10C8F00034464FF00109002E7AD0206D50B900BFA8
:10C90000502080F31188BFF34F8FBFF36F8F00BFAC
:10C9100000BFFEE7E06CB84201D23D4600E0E56CA6
:10C92000E06AA84264D0206D012861D131480068D6
:10C93000844201D0012000E0002050B900BF502007
:10C9400080F31188BFF34F8FBFF36F8F00BF00BF1D
:10C95000FEE7D4F82C80E562A06900F0004010B931
:10C96000C5F12000A06108EB8801234A02EB810198
:10C970006069884201D1012000E00020C0B3201D81
:10C98000FFF7E0FC40B994F82C10012088401B49C7
:10C99000096881431948016094F82C1001208840EF
:10C9A00016490968084315490860E16A01EB8101ED
:10C9B000114A02EB81014868A0608268E260211D93
:10C9C000826851608160E16A01EB81010A4A02EBF1
:10C9D00081026261E16A01EB8101074A52F821108C
:10C9E000491CE26A02EB8202034B43F8221000BFAB
:10C9F000BDE8F0876882FF1F84ADFF1F8082FF1FA4
:10CA00001CB51E4800210B468022CDE900101CA158
:10CA10001D4800F007FD0446012C02D101F062F828
:10CA20000446012C15D100BF502080F31188BFF3BC
:10CA30004F8FBFF36F8F00BF4FF0FF301349086077
:10CA400001201349086000201249086000F094F8A2
:10CA500010E0601C08B1012000E0002050B900BFC8
:10CA6000502080F31188BFF34F8FBFF36F8F00BF4B
:10CA700000BFFEE7084800681CBD00009C82FF1F45
:10CA800049444C45000000000DB500009882FF1F8E
:10CA90008482FF1F7C82FF1FA082FF1F0D4909684F
:10CAA00001440D4A1268914201D8012100E00021A1
:10CAB00051B900BF502181F31188BFF34F8FBFF3ED
:10CAC0006F8F00BF00BFFEE7024909680144014AB9
:10CAD000116070477C82FF1F9882FF1F0248006828
:10CAE000401C014908607047A482FF1F1D48006870
:10CAF00018B101201C49086032E000201A49086082
:10CB00001A480068B0FA80F0C0F11F0101EB810003
:10CB1000174A52F8200008B1012000E0002050B967
:10CB200000BF502080F31188BFF34F8FBFF36F8F8A
:10CB300000BF00BFFEE701EB81020D4B03EB82005B
:10CB400042685268426000F108024368934202D191
:10CB50004268526842604268D268064B1A6000BF61
:10CB600070470000A482FF1F8C82FF1F8082FF1F7E
:10CB700084ADFF1F6882FF1F1CB5524800685249F0
:10CB8000884201D0012000E0002050B900BF5020B1
:10CB900080F31188BFF34F8FBFF36F8F00BF00BFCB
:10CBA000FEE7484800684849491E884201D00120F4
:10CBB00000E0002050B900BF502080F31188BFF37F
:10CBC0004F8FBFF36F8F00BF00BFFEE73F4908469E
:10CBD00000780190FF200A46107008460078009007
:10CBE0009DF8000000F0F0009DF80020904201D177
:10CBF000012000E0002050B900BF502080F31188D0
:10CC0000BFF34F8FBFF36F8F00BF00BFFEE79DF8EC
:10CC1000000000F050002E4A107007202D4A1060CE
:10CC200009E02C480068401E2A4A10609DF8000068
:10CC30004006000E00909DF8000000F08000802863
:10CC4000EFD024480068C0F10700042801D101207A
:10CC500000E0002050B900BF502080F31188BFF3DE
:10CC60004F8FBFF36F8F00BF00BFFEE7194800680A
:10CC70000002184A10601046008800F4E06010605E
:10CC8000124A019810700F482030006840F470007C
:10CC90000C49203108600846006840F07040086088
:10CCA000FFF728FC00200C490860FBF7FFFA0B484F
:10CCB000006840F0404009490860FBF7E3FA0020B3
:10CCC0001CBD000000ED00E071C20F4100E400E077
:10CCD000EC82FF1FF082FF1FDC82FF1F34EF00E0B9
:10CCE0002DE9F84305460E4617460024E5B1601EBF
:10CCF000B0FBF5F0B04217D305FB06F010F1550F6D
:10CD000012D805FB06F808F15400FEF781FF04462F
:10CD1000B4B1A14609F154093B464A46314628467A
:10CD20000094FEF731FC0BE054B900BF502080F3B3
:10CD30001188BFF34F8FBFF36F8F00BF00BFFEE7B7
:10CD40002046BDE8F88300002DE9F04105460E4677
:10CD500001272C4654B900BF502080F31188BFF33F
:10CD60004F8FBFF36F8F00BF00BFFEE7002C42D094
:10CD7000E06B00283FD04FF0FF31E06BB1FBF0F0EB
:10CD8000216C884237D3FFF71BFBD4E90F122068D0
:10CD900001FB0200A0600020A06320686060E06BDF
:10CDA000401E226C216800FB0211E160FF2084F824
:10CDB000440084F845009EB9206908B9012000E0CC
:10CDC0000020A8B904F1100000F03EFD80B14FF042
:10CDD000805013490860BFF34F8FBFF36F8F07E098
:10CDE00004F11000FFF7C2FA04F12400FFF7BEFAC5
:10CDF000FFF710FB00E000270FB1012000E000204A
:10CE000050B900BF502080F31188BFF34F8FBFF39C
:10CE10006F8F00BF00BFFEE73846BDE8F08100001D
:10CE200004ED00E02DE9F84F80468B4615461E467E
:10CE3000444654B900BF502080F31188BFF34F8F90
:10CE4000BFF36F8F00BF00BFFEE7BBF1000F01D142
:10CE5000206C08B9012000E0002050B900BF50202C
:10CE600080F31188BFF34F8FBFF36F8F00BF00BFF8
:10CE7000FEE7022E02D1E06B012801D1012000E083
:10CE8000002050B900BF502080F31188BFF34F8FAE
:10CE9000BFF36F8F00BF00BFFEE7FFF705FC00BFC9
:10CEA0005021EFF3118081F31188BFF34F8FBFF34F
:10CEB0006F8F00BF0746A06BE16B884201D3022E43
:10CEC00042D194F945A0A06B0090324659462046C5
:10CED000FEF751FA0AF10100E0B9A06C58B1022E38
:10CEE00001D1009868BB2046FEF777FC48B345B3F4
:10CEF0000120286025E0606A08B9012000E00020D8
:10CF0000F8B904F1240000F09FFCD0B1CDB10120AC
:10CF1000286016E0BAF17F0F01D0012000E0002068
:10CF200050B900BF502080F31188BFF34F8FBFF37B
:10CF30006F8F00BF00BFFEE70AF1010040B284F826
:10CF400045004FF0010901E04FF0000900BF87F3F1
:10CF5000118800BF4846BDE8F88F2DE9F047074625
:10CF60000D463C4654B900BF502080F31188BFF3F2
:10CF70004F8FBFF36F8F00BF00BFFEE7206C08B973
:10CF8000012000E0002050B900BF502080F311883C
:10CF9000BFF34F8FBFF36F8F00BF00BFFEE7206866
:10CFA00008B9A06808B9012000E0002050B900BF0E
:10CFB000502080F31188BFF34F8FBFF36F8F00BFF6
:10CFC00000BFFEE7FFF770FB00BF5021EFF31180B9
:10CFD00081F31188BFF34F8FBFF36F8F00BF0646F9
:10CFE000D4F838A0E06B50453AD994F945900AF14D
:10CFF0000100A06309F10100C0B9A06C38B120465E
:10D00000FEF7EBFB48B345B30120286025E0606ADA
:10D0100008B9012000E00020F8B904F1240000F074
:10D0200013FCD0B1CDB10120286016E0B9F17F0F1B
:10D0300001D0012000E0002050B900BF502080F353
:10D040001188BFF34F8FBFF36F8F00BF00BFFEE7A4
:10D0500009F1010040B284F845004FF0010801E0F9
:10D060004FF0000800BF86F3118800BF4046BDE8BE
:10D07000F08700002DE9F74183B005460E464FF0DA
:10D0800000082C4654B900BF502080F31188BFF32C
:10D090004F8FBFF36F8F00BF00BFFEE70EB9206C4C
:10D0A00008B9012000E0002050B900BF502080F3F3
:10D0B0001188BFF34F8FBFF36F8F00BF00BFFEE734
:10D0C00000F0E0F908B9059808B9012000E0002057
:10D0D00050B900BF502080F31188BFF34F8FBFF3CA
:10D0E0006F8F00BF00BFFEE700BFFFF769F9A76BB6
:10D0F000F7B131462046FEF729F9781EA063206972
:10D1000008B9012000E0002060B904F1100000F02F
:10D110009BFB38B14FF080502F490860BFF34F8F11
:10D12000BFF36F8FFFF776F9012006B0BDE8F081FD
:10D13000059818B9FFF76EF90020F6E7B8F1000F6F
:10D1400004D101A8FFF770FB4FF00108FFF762F967
:10D15000FFF7C4FCFFF734F994F94400401C10B900
:10D16000002084F8440094F94500401C10B90020C8
:10D1700084F84500FFF74EF905A901A800F00AF967
:10D18000F0B92046FEF71CFBA0B104F1240005997C
:10D19000FFF75CFB2046FEF7F2FC00F0E7FB0028FF
:10D1A000A3D14FF080500C490860BFF34F8FBFF3FD
:10D1B0006F8F9AE72046FEF7E2FC00F0D7FB94E77A
:10D1C0002046FEF7DCFC00F0D1FB2046FEF7F8FA23
:10D1D00000288AD00020A8E704ED00E02DE9F34103
:10D1E00082B005464FF000082C46002654B900BF17
:10D1F000502080F31188BFF34F8FBFF36F8F00BFB4
:10D2000000BFFEE7206C08B9012000E0002050B903
:10D2100000BF502080F31188BFF34F8FBFF36F8F93
:10D2200000BF00BFFEE700F02DF908B9039808B968
:10D23000012000E0002050B900BF502080F3118889
:10D24000BFF34F8FBFF36F8F00BF00BFFEE700BF7C
:10D25000FFF7B6F8A76BFFB1781EA063206810B97E
:10D26000FEF78CFDA060206908B9012000E00020D5
:10D2700060B904F1100000F0E7FA38B14FF08050C7
:10D2800043490860BFF34F8FBFF36F8FFFF7C2F8BA
:10D29000012004B0BDE8F081039898B90EB90120CF
:10D2A00000E0002050B900BF502080F31188BFF388
:10D2B0004F8FBFF36F8F00BF00BFFEE7FFF7AAF8E5
:10D2C0000020E6E7B8F1000F04D16846FFF7ACFA9A
:10D2D0004FF00108FFF79EF8FFF700FCFFF770F82A
:10D2E00094F94400401C10B9002084F8440094F9DB
:10D2F0004500401C10B9002084F84500FFF78AF86B
:10D3000003A9684600F046F840BB2046FEF758FAED
:10D31000F0B1206838B9FFF753F8A06800F01EFAA2
:10D320000646FFF777F804F124000399FFF78EFA19
:10D330002046FEF724FC00F019FB002888D14FF0AE
:10D34000805013490860BFF34F8FBFF36F8F7FE7A3
:10D350002046FEF714FC00F009FB79E72046FEF7B3
:10D360000EFC00F003FB2046FEF72AFA0028EED060
:10D370005EB1FFF725F82046FEF745F80746394627
:10D38000A068FFF7B1FAFFF745F8002081E7000039
:10D3900004ED00E070B505460C4655B900BF5020BD
:10D3A00080F31188BFF34F8FBFF36F8F00BF00BFB3
:10D3B000FEE754B900BF502080F31188BFF34F8FB0
:10D3C000BFF36F8F00BF00BFFEE7FEF7F9FF134802
:10D3D00002686868131A2068401C08B9002619E022
:10D3E0000F4928680968884206D06868904203D8C7
:10D3F0000126002020600DE02068984207D92068AF
:10D40000C01A20602846FFF70FFA002602E000202D
:10D4100020600126FEF7FEFF304670BD7C82FF1FB4
:10D420009082FF1F2DE9FF4F85B080468946174641
:10D43000DDE912ABB800FEF7EBFB064656B15C2007
:10D44000FEF7E6FB04460CB1266304E03046FEF727
:10D45000FFFF00E000247CB10020CDE900ABCDE966
:10D4600002403A4649464046089BFEF7A4F820464B
:10D47000FDF7A0FE012501E04FF0FF35284609B079
:10D48000BDE8F08F0549096809B9012005E00449A4
:10D49000096809B9022000E0002070478482FF1F5C
:10D4A000A482FF1F01490868704700007C82FF1FAB
:10D4B0002DE9F0414FF000086148006800287DD157
:10D4C00060480068451C5F48056015BB5E48006801
:10D4D000006808B9012000E0002050B900BF5020CA
:10D4E00080F31188BFF34F8FBFF36F8F00BF00BF72
:10D4F000FEE7554807685548006853490860534897
:10D50000076053480068401C51490860FEF7BAFAAA
:10D5100000BF50480068854277D300BF4A48006882
:10D52000006808B9012000E0002020B14FF0FF3072
:10D530004849086068E044480068C068C468666894
:10D54000B54202D2434806605EE06069D4E9021247
:10D550008A60D4E902214A60211D42688A4201D1D1
:10D56000E1684160002262610168491E0160A06AB1
:10D5700098B1A06AD4E907128A60D4E907214A6009
:10D5800004F1180142688A4201D1216A41600022F7
:10D59000A2620168491E016000BF94F82C100120AE
:10D5A00088402D49096808432B490860E16A01EB6E
:10D5B00081012A4A02EB8101486800E037E0A0605F
:10D5C0008268E260211D826851608160E16A01EB3E
:10D5D0008101224A02EB81026261E16A01EB810171
:10D5E0001E4A52F82110491CE26A02EB82021B4BD0
:10D5F00043F822101A49E06A0968C96A88428DD343
:10D600004FF001088AE700E000BF15480068C06AD3
:10D6100000EB8000114951F82000012801D94FF09A
:10D6200001081048006808B14FF0010804E00E48F6
:10D630000068401C0C4908604046BDE8F0810000CD
:10D64000A482FF1F7C82FF1F6C82FF1F7082FF1F5E
:10D650009082FF1F9882FF1F8082FF1F84ADFF1FF3
:10D660006882FF1F8C82FF1F8882FF1F70B50546EE
:10D670002C460026002D68D035480068844201D130
:10D68000012000E0002050B900BF502080F3118835
:10D69000BFF34F8FBFF36F8F00BF00BFFEE7206D5A
:10D6A00050B900BF502080F31188BFF34F8FBFF3F4
:10D6B0006F8F00BF00BFFEE7206D401E2065E16C4C
:10D6C000E06A884241D0206D00283ED1201DFEF73F
:10D6D00039FE40B994F82C10012088401D49096892
:10D6E00081431C480160E06CE062E06AC0F1200008
:10D6F000A06194F82C10012088401649096808435D
:10D7000014490860E16A01EB8101134A02EB8101CF
:10D710004868A0608268E260211D82685160816073
:10D72000E16A01EB81010C4A02EB81026261E16A6C
:10D7300001EB8101084A52F82110491CE26A02EB10
:10D740008202054B43F822100126304670BD0000CE
:10D750006882FF1F8082FF1F84ADFF1F70B50546E2
:10D760002C460026002D67D03449E06A0968C96A52
:10D7700088425AD2A06900F0004028B92F480068BA
:10D78000C06AC0F12000A061E16A01EB81012C4A6E
:10D7900002EB81016069884201D1012000E0002094
:10D7A000E0B3201DFEF7CEFD40B994F82C10012007
:10D7B0008840244909688143224801601F48006865
:10D7C000C06AE06294F82C10012088401D49096865
:10D7D00008431C490860E16A01EB8101184A02EB29
:10D7E00081014868A0608268E260211D8268516002
:10D7F0008160E16A01EB8101114A02EB8102626101
:10D80000E16A01EB81010E4A52F82110491CE26ADB
:10D8100002EB82020A4B43F8221004E0FFE70748BC
:10D820000068C06AE062012606E00449E06C09680D
:10D83000C96A884200D20126304670BD6882FF1F47
:10D8400084ADFF1F8082FF1F70B50646F068C46874
:10D8500054B900BF502080F31188BFF34F8FBFF33E
:10D860006F8F00BF00BFFEE7A06AD4E907128A608D
:10D87000D4E907214A6004F1180142688A4201D1C3
:10D88000216A41600022A2620168491E016031489C
:10D89000006800283FD16069D4E902128A60D4E9A7
:10D8A00002214A60211D42688A4201D1E16841603B
:10D8B000002262610168491E016094F82C10012069
:10D8C000884025490968084323490860E16A01EB5B
:10D8D0008101224A02EB81014868A0608268E2600F
:10D8E000211D826851608160E16A01EB81011B4A60
:10D8F00002EB81026261E16A01EB8101174A52F891
:10D900002110491CE26A02EB8202144B43F82210F8
:10D91000FEF7B8F810E012494868E06182682262B8
:10D9200004F118018268516081600D4AA2621146BB
:10D930000968491C116000BF0A49E06A0968C96AA0
:10D94000884204D9012501200749086000E000252C
:10D95000284670BDA482FF1F8082FF1F84ADFF1F79
:10D960002CB0FF1F6882FF1F8C82FF1F70B5002440
:10D9700000265348006850B900BF502080F311883A
:10D98000BFF34F8FBFF36F8F00BF00BFFEE7FEF7FF
:10D9900017FD4B480068401E49490860084600686A
:10D9A00000287DD147480068002879D05BE04648D0
:10D9B000C068C468A06AD4E907128A60D4E9072164
:10D9C0004A6004F1180142688A4201D1216A41602B
:10D9D0000022A2620168491E01606069D4E9021256
:10D9E0008A60D4E902214A60211D42688A4201D13D
:10D9F000E1684160002262610168491E016094F89B
:10DA00002C10012088403149096808432F490860DB
:10DA1000E16A01EB81012E4A02EB81014868A060B6
:10DA20008268E260211D826851608160E16A01EBD9
:10DA30008101274A02EB81026261E16A01EB810107
:10DA4000234A52F82110491CE26A02EB8202204B61
:10DA500043F822101F49E06A0968C96A884202D364
:10DA600001201D4908601848006808B9012000E03D
:10DA7000002000289BD00CB1FEF704F81748056879
:10DA800065B100BFFFF714FD10B101201249086015
:10DA90006D1E002DF6D10020104908600E4800E0F0
:10DAA00009E0006838B1012630070D490860BFF36E
:10DAB0004F8FBFF36F8FFEF7ADFC304670BD000097
:10DAC000A482FF1F7882FF1F2CB0FF1F8082FF1FE0
:10DAD00084ADFF1F6882FF1F8C82FF1F8882FF1F9B
:10DAE00004ED00E01CB50024FDF7DAFB0D480068EA
:10DAF00050B10D4802210023CA01CDE900100BA14D
:10DB00000C48FFF78FFC044654B900BF502080F347
:10DB10001188BFF34F8FBFF36F8F00BF00BFFEE7C9
:10DB200020461CBDB082FF1FB482FF1F546D7220BF
:10DB30005376630065BB00006173646173643030C9
:10DB400000000000000000000000000000000000D5
:10DB500000000000000000000000000000000000C5
:10DB600000000000000000000000000000000000B5
:10DB700000000000000000000000000000000000A5
:10DB80000000000000000000000000000000000095
:10DB90000000000000000000000000000000000085
:10DBA0000000000000000000000000000000000075
:10DBB0000000000000000000000000000000000065
:10DBC0000000000000000000000000000000000055
:10DBD0000000000000000000000000000000000045
:10DBE0000000000000000000000000000000000035
:10DBF0000000000000000000000000000000000025
:10DC00000000000000000000000000000000000014
:10DC10000000000000000000000000000000000004
:10DC200000000000000000000000000000000000F4
:10DC300000000000000000000001020304050607C8
:10DC4000080C1014182030401014181C20283848D4
:10DC500070DC00000080FF1FFC0200005484000004
:10DC600084DE0000FC82FF1F9CB40000E89C0000E2
:10DC70003120ED5E36BC6CE25A78D926EFC4B59AF5
:10DC80008389FFD7C935936BA5F126AF104D4A1391
:10DC90007C6BB23584D7DE89E8136B4D5DAF07F13D
:10DCA00031E24DBC7B5E2100179A94C4A226F8781D
:10DCB000CEAF29F11F13454D73D7F089C66B9C3544
:10DCC000AA26D678E09ABAC48C5E0F0039E263BC0B
:10DCD00055C49B9AAD78F726C1BC42E274002E5E13
:10DCE000184D641352F108AF3E35BD6B8B89D1D707
:10DCF000E75E530065E23FBC09268A78BC9AE6C419
:10DD0000D0D7AC899A6BC035F6AF75F14313194D76
:10DD10002F35E16BD7898DD7BB4D38130EF154AF3A
:10DD200062BC1EE22800725E44C4C79AF178AB263A
:10DD30009DF17AAF4C4D16132089A3D79535CF6B43
:10DD4000F9788526B3C4E99ADF005C5E6ABC30E2EC
:10DD5000069AC8C4FE26A47892E211BC275E7D20F4
:10DD6000FC4B13374D01AF5BF16D6BEE35D8D782AD
:10DD700089B4BCA6E29000CA5EFCC47F9A497813BD
:10DD8000262535596B6F8935D7034D8013B6F1ECD5
:10DD9000AFDAD71489226B78354EAFCDF1FB13A1E2
:10DDA0004D975EEB00DDE287BCB1263278049A5EC7
:10DDB000C468138F4DB9AFE3F1D56B563560D73AD0
:10DDC000890C9A70C446261C782AE2A9BC9F5EC5BD
:10DDD00000F3783D260BC4519A6700E45ED2BC88FC
:10DDE000E2BEF1C2AFF44DAE1398891BD72D357743
:10DDF0006B41E2F5BCC35E9900AF9A2CC41A264071
:10DE000078766B0A353CD766895013D34DE5AFBFA2
:10DE1000F1898947D771352B6B1DF19EAFA84DF263
:10DE200013C400B85E8EBCD4E2E278612657C40DFC
:10DE30009A3B4DDC13EAF1B0AF8635056B33896947
:10DE4000D75FC4239A15784F2679BCFAE2CC0096A6
:10DE50005EA0266E78589A02C4345EB700165181CF
:10DE6000E2DBBCEDAF91F1A713FD4DCBD748897E26
:10DE70006B243512F3BE15024001023C1F051DAA9A
:04DE8000AAAAAA00A0
:040000050000825124
:00000001FF
